 instrument

 Timestamp is 82fc8020 (reproducible build file hash)

 Preferred load address is 0000000180000000

 Start         Length     Name                   Class
 0001:00000000 00005dc0H .text$mn                CODE
 0001:00005dc0 00000036H .text$mn$00             CODE
 0001:00005df6 00000092H .text$x                 CODE
 0002:00000000 000001d8H .idata$5                DATA
 0002:000001d8 00000038H .00cfg                  DATA
 0002:00000210 00000008H .CRT$XCA                DATA
 0002:00000218 00000008H .CRT$XCZ                DATA
 0002:00000220 00000008H .CRT$XIA                DATA
 0002:00000228 00000008H .CRT$XIZ                DATA
 0002:00000230 00000008H .CRT$XPA                DATA
 0002:00000238 00000008H .CRT$XPZ                DATA
 0002:00000240 00000008H .CRT$XTA                DATA
 0002:00000248 00000008H .CRT$XTZ                DATA
 0002:00000250 00000000H .gehcont$y              DATA
 0002:00000250 00000000H .gfids$y                DATA
 0002:00000250 00001a30H .rdata                  DATA
 0002:00001c80 00000000H .rdata$CastGuardVftablesA DATA
 0002:00001c80 00000000H .rdata$CastGuardVftablesC DATA
 0002:00001c80 0000006cH .rdata$voltmd           DATA
 0002:00001cec 000002bcH .rdata$zzzdbg           DATA
 0002:00001fa8 00000008H .rtc$IAA                DATA
 0002:00001fb0 00000008H .rtc$IZZ                DATA
 0002:00001fb8 00000008H .rtc$TAA                DATA
 0002:00001fc0 00000008H .rtc$TZZ                DATA
 0002:00001fc8 000004e8H .xdata                  DATA
 0002:000024b0 00000418H .edata                  DATA
 0002:000028c8 000000c8H .idata$2                DATA
 0002:00002990 00000018H .idata$3                DATA
 0002:000029a8 000001d8H .idata$4                DATA
 0002:00002b80 00000488H .idata$6                DATA
 0003:00000000 00000040H .data                   DATA
 0003:00000040 00000618H .bss                    DATA
 0004:00000000 000005a0H .pdata                  DATA
 0005:00000000 00000060H .rsrc$01                DATA
 0005:00000060 00000340H .rsrc$02                DATA

  Address         Publics by Value              Rva+Base               Lib:Object

 0000:00000000       __AbsoluteZero             0000000000000000     <absolute>
 0000:00000000       ___safe_se_handler_count   0000000000000000     <absolute>
 0000:00000000       ___safe_se_handler_table   0000000000000000     <absolute>
 0000:00000000       __arm64x_extra_rfe_table   0000000000000000     <absolute>
 0000:00000000       __arm64x_extra_rfe_table_size 0000000000000000     <absolute>
 0000:00000000       __arm64x_native_entrypoint 0000000000000000     <absolute>
 0000:00000000       __arm64x_redirection_metadata 0000000000000000     <absolute>
 0000:00000000       __arm64x_redirection_metadata_count 0000000000000000     <absolute>
 0000:00000000       __dynamic_value_reloc_table 0000000000000000     <absolute>
 0000:00000000       __enclave_config           0000000000000000     <absolute>
 0000:00000000       __guard_check_icall_a64n_fptr 0000000000000000     <absolute>
 0000:00000000       __guard_eh_cont_count      0000000000000000     <absolute>
 0000:00000000       __guard_eh_cont_table      0000000000000000     <absolute>
 0000:00000000       __guard_fids_count         0000000000000000     <absolute>
 0000:00000000       __guard_fids_table         0000000000000000     <absolute>
 0000:00000000       __guard_iat_count          0000000000000000     <absolute>
 0000:00000000       __guard_iat_table          0000000000000000     <absolute>
 0000:00000000       __guard_longjmp_count      0000000000000000     <absolute>
 0000:00000000       __guard_longjmp_table      0000000000000000     <absolute>
 0000:00000000       __hybrid_auxiliary_delayload_iat 0000000000000000     <absolute>
 0000:00000000       __hybrid_auxiliary_delayload_iat_copy 0000000000000000     <absolute>
 0000:00000000       __hybrid_auxiliary_iat     0000000000000000     <absolute>
 0000:00000000       __hybrid_auxiliary_iat_copy 0000000000000000     <absolute>
 0000:00000000       __hybrid_code_map          0000000000000000     <absolute>
 0000:00000000       __hybrid_code_map_count    0000000000000000     <absolute>
 0000:00000000       __hybrid_image_info_bitfield 0000000000000000     <absolute>
 0000:00000000       __x64_code_ranges_to_entry_points 0000000000000000     <absolute>
 0000:00000000       __x64_code_ranges_to_entry_points_count 0000000000000000     <absolute>
 0000:00000100       __guard_flags              0000000000000100     <absolute>
 0000:00000000       __ImageBase                0000000180000000     <linker-defined>
 0001:00000000       convertUtf8ToModifiedUtf8  0000000180001000 f   EncodingSupport.obj
 0001:00000178       modifiedUtf8LengthOfUtf8   0000000180001178 f   EncodingSupport.obj
 0001:00000278       convertUtf8ToPlatformString 0000000180001278 f   EncodingSupport_md.obj
 0001:00000394       __local_stdio_printf_options 0000000180001394 f i FileSystemSupport_md.obj
 0001:0000039c       basePath                   000000018000139c f   FileSystemSupport_md.obj
 0001:00000448       fprintf                    0000000180001448 f i FileSystemSupport_md.obj
 0001:0000048c       fromURIPath                000000018000148c f   FileSystemSupport_md.obj
 0001:00000550       isAbsolute                 0000000180001550 f   FileSystemSupport_md.obj
 0001:00000764       normalize_path             0000000180001764 f   FileSystemSupport_md.obj
 0001:000007ec       resolve                    00000001800017ec f   FileSystemSupport_md.obj
 0001:00000964       Java_sun_instrument_InstrumentationImpl_appendToClassLoaderSearch0 0000000180001964 f   InstrumentationImplNativeMethods.obj
 0001:00000978       Java_sun_instrument_InstrumentationImpl_getAllLoadedClasses0 0000000180001978 f   InstrumentationImplNativeMethods.obj
 0001:00000980       Java_sun_instrument_InstrumentationImpl_getInitiatedClasses0 0000000180001980 f   InstrumentationImplNativeMethods.obj
 0001:0000098c       Java_sun_instrument_InstrumentationImpl_getObjectSize0 000000018000198c f   InstrumentationImplNativeMethods.obj
 0001:00000998       Java_sun_instrument_InstrumentationImpl_isModifiableClass0 0000000180001998 f   InstrumentationImplNativeMethods.obj
 0001:000009a4       Java_sun_instrument_InstrumentationImpl_isRetransformClassesSupported0 00000001800019a4 f   InstrumentationImplNativeMethods.obj
 0001:000009ac       Java_sun_instrument_InstrumentationImpl_jarFile 00000001800019ac f   InstrumentationImplNativeMethods.obj
 0001:000009b4       Java_sun_instrument_InstrumentationImpl_loadAgent0 00000001800019b4 f   InstrumentationImplNativeMethods.obj
 0001:000009e8       Java_sun_instrument_InstrumentationImpl_redefineClasses0 00000001800019e8 f   InstrumentationImplNativeMethods.obj
 0001:000009f4       Java_sun_instrument_InstrumentationImpl_retransformClasses0 00000001800019f4 f   InstrumentationImplNativeMethods.obj
 0001:00000a00       Java_sun_instrument_InstrumentationImpl_setHasRetransformableTransformers 0000000180001a00 f   InstrumentationImplNativeMethods.obj
 0001:00000a0c       Java_sun_instrument_InstrumentationImpl_setHasTransformers 0000000180001a0c f   InstrumentationImplNativeMethods.obj
 0001:00000a18       Java_sun_instrument_InstrumentationImpl_setNativeMethodPrefixes 0000000180001a18 f   InstrumentationImplNativeMethods.obj
 0001:00000a2c       Agent_OnAttach             0000000180001a2c f   InvocationAdapter.obj
 0001:00000dbc       Agent_OnLoad               0000000180001dbc f   InvocationAdapter.obj
 0001:00001084       Agent_OnUnload             0000000180002084 f   InvocationAdapter.obj
 0001:00001084       _guard_check_icall_nop     0000000180002084 f   MSVCRT:guard_support.obj
 0001:000015ac       convertCapabilityAttributes 00000001800025ac f   InvocationAdapter.obj
 0001:00001630       eventHandlerClassFileLoadHook 0000000180002630 f   InvocationAdapter.obj
 0001:000016f4       eventHandlerVMInit         00000001800026f4 f   InvocationAdapter.obj
 0001:000017c0       getBooleanAttribute        00000001800027c0 f   InvocationAdapter.obj
 0001:000017f0       loadAgent                  00000001800027f0 f   InvocationAdapter.obj
 0001:00001ac0       addNativeMethodPrefixCapability 0000000180002ac0 f   JPLISAgent.obj
 0001:00001af8       addOriginalMethodOrderCapability 0000000180002af8 f   JPLISAgent.obj
 0001:00001b90       addRedefineClassesCapability 0000000180002b90 f   JPLISAgent.obj
 0001:00001c5c       appendToClassLoaderSearch  0000000180002c5c f   JPLISAgent.obj
 0001:00001d98       checkCapabilities          0000000180002d98 f   JPLISAgent.obj
 0001:00001e34       commandStringIntoJavaStrings 0000000180002e34 f   JPLISAgent.obj
 0001:00001f10       commonGetClassList         0000000180002f10 f   JPLISAgent.obj
 0001:00001fe8       createInstrumentationImpl  0000000180002fe8 f   JPLISAgent.obj
 0001:000022e4       createNewJPLISAgent        00000001800032e4 f   JPLISAgent.obj
 0001:000023b4       deallocateCommandLineData  00000001800033b4 f   JPLISAgent.obj
 0001:000023e8       enableNativeMethodPrefixCapability 00000001800033e8 f   JPLISAgent.obj
 0001:00002478       getAllLoadedClasses        0000000180003478 f   JPLISAgent.obj
 0001:00002488       getAllLoadedClassesClassListFetcher 0000000180003488 f   JPLISAgent.obj
 0001:00002498       getInitiatedClasses        0000000180003498 f   JPLISAgent.obj
 0001:000024a4       getInitiatedClassesClassListFetcher 00000001800034a4 f   JPLISAgent.obj
 0001:000024b0       getJPLISEnvironment        00000001800034b0 f   JPLISAgent.obj
 0001:0000265c       getObjectArrayFromClasses  000000018000365c f   JPLISAgent.obj
 0001:00002768       getObjectSize              0000000180003768 f   JPLISAgent.obj
 0001:000027ec       initializeJPLISAgent       00000001800037ec f   JPLISAgent.obj
 0001:00002994       invokeJavaAgentMainMethod  0000000180003994 f   JPLISAgent.obj
 0001:00002a64       isModifiableClass          0000000180003a64 f   JPLISAgent.obj
 0001:00002ab8       isRetransformClassesSupported 0000000180003ab8 f   JPLISAgent.obj
 0001:00002abc       jarFile                    0000000180003abc f   JPLISAgent.obj
 0001:00002acc       processJavaStart           0000000180003acc f   JPLISAgent.obj
 0001:00002be4       recordCommandLineData      0000000180003be4 f   JPLISAgent.obj
 0001:00002cac       redefineClassMapper        0000000180003cac f   JPLISAgent.obj
 0001:00002d7c       redefineClasses            0000000180003d7c f   JPLISAgent.obj
 0001:000031f4       retransformClasses         00000001800041f4 f   JPLISAgent.obj
 0001:00003410       retransformableEnvironment 0000000180004410 f   JPLISAgent.obj
 0001:000035d0       setHasRetransformableTransformers 00000001800045d0 f   JPLISAgent.obj
 0001:00003650       setHasTransformers         0000000180004650 f   JPLISAgent.obj
 0001:000036c8       setLivePhaseEventHandlers  00000001800046c8 f   JPLISAgent.obj
 0001:00003788       setNativeMethodPrefixes    0000000180004788 f   JPLISAgent.obj
 0001:00003a88       startJavaAgent             0000000180004a88 f   JPLISAgent.obj
 0001:00003b4c       transformClassFile         0000000180004b4c f   JPLISAgent.obj
 0001:00003ea4       JPLISAssertCondition       0000000180004ea4 f   JPLISAssert.obj
 0001:00003ef4       JPLISAssertConditionWithMessage 0000000180004ef4 f   JPLISAssert.obj
 0001:0000403c       freeAttributes             000000018000503c f   JarFacade.obj
 0001:00004084       getAttribute               0000000180005084 f   JarFacade.obj
 0001:000040c8       readAttributes             00000001800050c8 f   JarFacade.obj
 0001:00004138       checkForAndClearThrowable  0000000180005138 f   JavaExceptions.obj
 0001:00004170       checkForThrowable          0000000180005170 f   JavaExceptions.obj
 0001:0000417c       createAndThrowInternalError 000000018000517c f   JavaExceptions.obj
 0001:000041b0       createAndThrowThrowableFromJVMTIErrorCode 00000001800051b0 f   JavaExceptions.obj
 0001:000041dc       createInternalError        00000001800051dc f   JavaExceptions.obj
 0001:000041ec       createThrowable            00000001800051ec f   JavaExceptions.obj
 0001:00004364       createThrowableFromJVMTIErrorCode 0000000180005364 f   JavaExceptions.obj
 0001:0000451c       getMessageFromThrowable    000000018000551c f   JavaExceptions.obj
 0001:00004668       initializeFallbackError    0000000180005668 f   JavaExceptions.obj
 0001:000046ec       isSafeForJNICalls          00000001800056ec f   JavaExceptions.obj
 0001:00004704       isUnchecked                0000000180005704 f   JavaExceptions.obj
 0001:000047b0       logThrowable               00000001800057b0 f   JavaExceptions.obj
 0001:000047d8       mapAllCheckedToInternalErrorMapper 00000001800057d8 f   JavaExceptions.obj
 0001:000048b4       mapThrownThrowableIfNecessary 00000001800058b4 f   JavaExceptions.obj
 0001:00004910       preserveThrowable          0000000180005910 f   JavaExceptions.obj
 0001:00004948       restoreThrowable           0000000180005948 f   JavaExceptions.obj
 0001:00004950       throwThrowable             0000000180005950 f   JavaExceptions.obj
 0001:00004b5c       validatePathChars          0000000180005b5c f   PathCharsValidator.obj
 0001:00004c5c       assertTLSValue             0000000180005c5c f   Reentrancy.obj
 0001:00004cc8       confirmingTLSSet           0000000180005cc8 f   Reentrancy.obj
 0001:00004d20       releaseReentrancyToken     0000000180005d20 f   Reentrancy.obj
 0001:00004d78       tryToAcquireReentrancyToken 0000000180005d78 f   Reentrancy.obj
 0001:00004e3c       abortJVM                   0000000180005e3c f   Utilities.obj
 0001:00004e48       allocate                   0000000180005e48 f   Utilities.obj
 0001:00004e9c       deallocate                 0000000180005e9c f   Utilities.obj
 0001:00004ed8       isInstanceofClassName      0000000180005ed8 f   Utilities.obj
 0001:00004fd4       JDK_Canonicalize           0000000180005fd4 f   java:java.dll
 0001:00004fda       JLI_ManifestIterate        0000000180005fda f   jli:jli.dll
 0001:00004fe0       JVM_PrintWarningAtDynamicAgentLoad 0000000180005fe0 f   jvm:jvm.dll
 0001:00004fe8       __GSHandlerCheck           0000000180005fe8 f   MSVCRT:gshandler.obj
 0001:00005008       __GSHandlerCheckCommon     0000000180006008 f   MSVCRT:gshandler.obj
 0001:00005080       __security_check_cookie    0000000180006080 f   MSVCRT:amdsecgs.obj
 0001:000053c0       _DllMainCRTStartup         00000001800063c0 f   MSVCRT:dll_dllmain.obj
 0001:00005400       __raise_securityfailure    0000000180006400 f   MSVCRT:gs_report.obj
 0001:00005434       __report_gsfailure         0000000180006434 f   MSVCRT:gs_report.obj
 0001:0000557c       __security_init_cookie     000000018000657c f   MSVCRT:gs_support.obj
 0001:00005628       DllMain                    0000000180006628 f   MSVCRT:dll_dllmain_stub.obj
 0001:0000564c       ?__scrt_initialize_type_info@@YAXXZ 000000018000664c f   MSVCRT:tncleanup.obj
 0001:0000565c       ?__scrt_uninitialize_type_info@@YAXXZ 000000018000665c f   MSVCRT:tncleanup.obj
 0001:00005668       __local_stdio_scanf_options 0000000180006668 f i MSVCRT:default_local_stdio_options.obj
 0001:00005670       __scrt_initialize_default_local_stdio_options 0000000180006670 f   MSVCRT:default_local_stdio_options.obj
 0001:0000568c       __scrt_acquire_startup_lock 000000018000668c f   MSVCRT:utility.obj
 0001:000056c8       __scrt_dllmain_after_initialize_c 00000001800066c8 f   MSVCRT:utility.obj
 0001:000056fc       __scrt_dllmain_before_initialize_c 00000001800066fc f   MSVCRT:utility.obj
 0001:00005714       __scrt_dllmain_crt_thread_attach 0000000180006714 f   MSVCRT:utility.obj
 0001:0000573c       __scrt_dllmain_crt_thread_detach 000000018000673c f   MSVCRT:utility.obj
 0001:00005754       __scrt_dllmain_exception_filter 0000000180006754 f   MSVCRT:utility.obj
 0001:000057b4       __scrt_dllmain_uninitialize_c 00000001800067b4 f   MSVCRT:utility.obj
 0001:000057e4       __scrt_dllmain_uninitialize_critical 00000001800067e4 f   MSVCRT:utility.obj
 0001:000057f8       __scrt_initialize_crt      00000001800067f8 f   MSVCRT:utility.obj
 0001:00005844       __scrt_initialize_onexit_tables 0000000180006844 f   MSVCRT:utility.obj
 0001:000058d0       __scrt_is_nonwritable_in_current_image 00000001800068d0 f   MSVCRT:utility.obj
 0001:00005968       __scrt_release_startup_lock 0000000180006968 f   MSVCRT:utility.obj
 0001:0000598c       __scrt_uninitialize_crt    000000018000698c f   MSVCRT:utility.obj
 0001:000059b8       __scrt_get_dyn_tls_init_callback 00000001800069b8 f   MSVCRT:dyn_tls_init.obj
 0001:000059c0       __crt_debugger_hook        00000001800069c0 f   MSVCRT:utility_desktop.obj
 0001:000059c8       __scrt_fastfail            00000001800069c8 f   MSVCRT:utility_desktop.obj
 0001:00005b14       _RTC_Initialize            0000000180006b14 f   MSVCRT:initsect.obj
 0001:00005b50       _RTC_Terminate             0000000180006b50 f   MSVCRT:initsect.obj
 0001:00005b8c       __isa_available_init       0000000180006b8c f   MSVCRT:cpu_disp.obj
 0001:00005d38       _get_startup_argv_mode     0000000180006d38 f   MSVCRT:argv_mode.obj
 0001:00005d40       __scrt_is_ucrt_dll_in_use  0000000180006d40 f   MSVCRT:ucrt_detection.obj
 0001:00005d50       memcpy                     0000000180006d50 f   vcruntime:VCRUNTIME140.dll
 0001:00005d56       strchr                     0000000180006d56 f   vcruntime:VCRUNTIME140.dll
 0001:00005d5c       memset                     0000000180006d5c f   vcruntime:VCRUNTIME140.dll
 0001:00005d62       strrchr                    0000000180006d62 f   vcruntime:VCRUNTIME140.dll
 0001:00005d68       __C_specific_handler       0000000180006d68 f   vcruntime:VCRUNTIME140.dll
 0001:00005d6e       __std_type_info_destroy_list 0000000180006d6e f   vcruntime:VCRUNTIME140.dll
 0001:00005d74       strlen                     0000000180006d74 f   ucrt:api-ms-win-crt-string-l1-1-0.dll
 0001:00005d7a       strcpy                     0000000180006d7a f   ucrt:api-ms-win-crt-string-l1-1-0.dll
 0001:00005d80       _initterm                  0000000180006d80 f   ucrt:api-ms-win-crt-runtime-l1-1-0.dll
 0001:00005d86       _initterm_e                0000000180006d86 f   ucrt:api-ms-win-crt-runtime-l1-1-0.dll
 0001:00005d8c       _seh_filter_dll            0000000180006d8c f   ucrt:api-ms-win-crt-runtime-l1-1-0.dll
 0001:00005d92       _configure_narrow_argv     0000000180006d92 f   ucrt:api-ms-win-crt-runtime-l1-1-0.dll
 0001:00005d98       _initialize_narrow_environment 0000000180006d98 f   ucrt:api-ms-win-crt-runtime-l1-1-0.dll
 0001:00005d9e       _initialize_onexit_table   0000000180006d9e f   ucrt:api-ms-win-crt-runtime-l1-1-0.dll
 0001:00005da4       _execute_onexit_table      0000000180006da4 f   ucrt:api-ms-win-crt-runtime-l1-1-0.dll
 0001:00005daa       _cexit                     0000000180006daa f   ucrt:api-ms-win-crt-runtime-l1-1-0.dll
 0001:00005db0       __acrt_initialize          0000000180006db0 f   MSVCRT:ucrt_stubs.obj
 0001:00005db0       __acrt_thread_attach       0000000180006db0 f   MSVCRT:ucrt_stubs.obj
 0001:00005db0       __acrt_thread_detach       0000000180006db0 f   MSVCRT:ucrt_stubs.obj
 0001:00005db0       __acrt_uninitialize        0000000180006db0 f   MSVCRT:ucrt_stubs.obj
 0001:00005db0       __acrt_uninitialize_critical 0000000180006db0 f   MSVCRT:ucrt_stubs.obj
 0001:00005db0       __scrt_stub_for_acrt_initialize 0000000180006db0 f   MSVCRT:ucrt_stubs.obj
 0001:00005db0       __scrt_stub_for_acrt_thread_attach 0000000180006db0 f   MSVCRT:ucrt_stubs.obj
 0001:00005db0       __scrt_stub_for_acrt_thread_detach 0000000180006db0 f   MSVCRT:ucrt_stubs.obj
 0001:00005db0       __scrt_stub_for_acrt_uninitialize 0000000180006db0 f   MSVCRT:ucrt_stubs.obj
 0001:00005db0       __scrt_stub_for_acrt_uninitialize_critical 0000000180006db0 f   MSVCRT:ucrt_stubs.obj
 0001:00005db0       __vcrt_initialize          0000000180006db0 f   MSVCRT:ucrt_stubs.obj
 0001:00005db0       __vcrt_thread_attach       0000000180006db0 f   MSVCRT:ucrt_stubs.obj
 0001:00005db0       __vcrt_thread_detach       0000000180006db0 f   MSVCRT:ucrt_stubs.obj
 0001:00005db0       __vcrt_uninitialize        0000000180006db0 f   MSVCRT:ucrt_stubs.obj
 0001:00005db0       __vcrt_uninitialize_critical 0000000180006db0 f   MSVCRT:ucrt_stubs.obj
 0001:00005db4       __scrt_stub_for_is_c_termination_complete 0000000180006db4 f   MSVCRT:ucrt_stubs.obj
 0001:00005db4       _is_c_termination_complete 0000000180006db4 f   MSVCRT:ucrt_stubs.obj
 0001:00005dd0       _guard_dispatch_icall_nop  0000000180006dd0 f   MSVCRT:guard_dispatch.obj
 0001:00005df0       _guard_xfg_dispatch_icall_nop 0000000180006df0 f   MSVCRT:guard_xfg_dispatch.obj
 0002:00000000       __imp_IsDebuggerPresent    0000000180007000     kernel32:KERNEL32.dll
 0002:00000008       __imp_InitializeSListHead  0000000180007008     kernel32:KERNEL32.dll
 0002:00000010       __imp_DisableThreadLibraryCalls 0000000180007010     kernel32:KERNEL32.dll
 0002:00000018       __imp_GetSystemTimeAsFileTime 0000000180007018     kernel32:KERNEL32.dll
 0002:00000020       __imp_MultiByteToWideChar  0000000180007020     kernel32:KERNEL32.dll
 0002:00000028       __imp_WideCharToMultiByte  0000000180007028     kernel32:KERNEL32.dll
 0002:00000030       __imp_GetACP               0000000180007030     kernel32:KERNEL32.dll
 0002:00000038       __imp_GetLocaleInfoA       0000000180007038     kernel32:KERNEL32.dll
 0002:00000040       __imp_GetUserDefaultLCID   0000000180007040     kernel32:KERNEL32.dll
 0002:00000048       __imp_RtlCaptureContext    0000000180007048     kernel32:KERNEL32.dll
 0002:00000050       __imp_RtlLookupFunctionEntry 0000000180007050     kernel32:KERNEL32.dll
 0002:00000058       __imp_RtlVirtualUnwind     0000000180007058     kernel32:KERNEL32.dll
 0002:00000060       __imp_UnhandledExceptionFilter 0000000180007060     kernel32:KERNEL32.dll
 0002:00000068       __imp_SetUnhandledExceptionFilter 0000000180007068     kernel32:KERNEL32.dll
 0002:00000070       __imp_GetCurrentProcess    0000000180007070     kernel32:KERNEL32.dll
 0002:00000078       __imp_TerminateProcess     0000000180007078     kernel32:KERNEL32.dll
 0002:00000080       __imp_IsProcessorFeaturePresent 0000000180007080     kernel32:KERNEL32.dll
 0002:00000088       __imp_QueryPerformanceCounter 0000000180007088     kernel32:KERNEL32.dll
 0002:00000090       __imp_GetCurrentProcessId  0000000180007090     kernel32:KERNEL32.dll
 0002:00000098       __imp_GetCurrentThreadId   0000000180007098     kernel32:KERNEL32.dll
 0002:000000a0       \177KERNEL32_NULL_THUNK_DATA 00000001800070a0     kernel32:KERNEL32.dll
 0002:000000a8       __imp___std_type_info_destroy_list 00000001800070a8     vcruntime:VCRUNTIME140.dll
 0002:000000b0       __imp___C_specific_handler 00000001800070b0     vcruntime:VCRUNTIME140.dll
 0002:000000b8       __imp_strrchr              00000001800070b8     vcruntime:VCRUNTIME140.dll
 0002:000000c0       __imp_memset               00000001800070c0     vcruntime:VCRUNTIME140.dll
 0002:000000c8       __imp_memcpy               00000001800070c8     vcruntime:VCRUNTIME140.dll
 0002:000000d0       __imp_strchr               00000001800070d0     vcruntime:VCRUNTIME140.dll
 0002:000000d8       \177VCRUNTIME140_NULL_THUNK_DATA 00000001800070d8     vcruntime:VCRUNTIME140.dll
 0002:000000e0       __imp_atoi                 00000001800070e0     ucrt:api-ms-win-crt-convert-l1-1-0.dll
 0002:000000e8       \177api-ms-win-crt-convert-l1-1-0_NULL_THUNK_DATA 00000001800070e8     ucrt:api-ms-win-crt-convert-l1-1-0.dll
 0002:000000f0       __imp_free                 00000001800070f0     ucrt:api-ms-win-crt-heap-l1-1-0.dll
 0002:000000f8       __imp_realloc              00000001800070f8     ucrt:api-ms-win-crt-heap-l1-1-0.dll
 0002:00000100       __imp_calloc               0000000180007100     ucrt:api-ms-win-crt-heap-l1-1-0.dll
 0002:00000108       __imp_malloc               0000000180007108     ucrt:api-ms-win-crt-heap-l1-1-0.dll
 0002:00000110       \177api-ms-win-crt-heap-l1-1-0_NULL_THUNK_DATA 0000000180007110     ucrt:api-ms-win-crt-heap-l1-1-0.dll
 0002:00000118       __imp__seh_filter_dll      0000000180007118     ucrt:api-ms-win-crt-runtime-l1-1-0.dll
 0002:00000120       __imp__execute_onexit_table 0000000180007120     ucrt:api-ms-win-crt-runtime-l1-1-0.dll
 0002:00000128       __imp__initialize_onexit_table 0000000180007128     ucrt:api-ms-win-crt-runtime-l1-1-0.dll
 0002:00000130       __imp__cexit               0000000180007130     ucrt:api-ms-win-crt-runtime-l1-1-0.dll
 0002:00000138       __imp__initialize_narrow_environment 0000000180007138     ucrt:api-ms-win-crt-runtime-l1-1-0.dll
 0002:00000140       __imp__initterm            0000000180007140     ucrt:api-ms-win-crt-runtime-l1-1-0.dll
 0002:00000148       __imp__initterm_e          0000000180007148     ucrt:api-ms-win-crt-runtime-l1-1-0.dll
 0002:00000150       __imp__configure_narrow_argv 0000000180007150     ucrt:api-ms-win-crt-runtime-l1-1-0.dll
 0002:00000158       \177api-ms-win-crt-runtime-l1-1-0_NULL_THUNK_DATA 0000000180007158     ucrt:api-ms-win-crt-runtime-l1-1-0.dll
 0002:00000160       __imp___acrt_iob_func      0000000180007160     ucrt:api-ms-win-crt-stdio-l1-1-0.dll
 0002:00000168       __imp___stdio_common_vfprintf 0000000180007168     ucrt:api-ms-win-crt-stdio-l1-1-0.dll
 0002:00000170       \177api-ms-win-crt-stdio-l1-1-0_NULL_THUNK_DATA 0000000180007170     ucrt:api-ms-win-crt-stdio-l1-1-0.dll
 0002:00000178       __imp_strlen               0000000180007178     ucrt:api-ms-win-crt-string-l1-1-0.dll
 0002:00000180       __imp__stricmp             0000000180007180     ucrt:api-ms-win-crt-string-l1-1-0.dll
 0002:00000180       __imp_stricmp              0000000180007180     ucrt:api-ms-win-crt-string-l1-1-0.dll
 0002:00000188       __imp_strcpy               0000000180007188     ucrt:api-ms-win-crt-string-l1-1-0.dll
 0002:00000190       __imp_strncpy              0000000180007190     ucrt:api-ms-win-crt-string-l1-1-0.dll
 0002:00000198       __imp__strdup              0000000180007198     ucrt:api-ms-win-crt-string-l1-1-0.dll
 0002:00000198       __imp_strdup               0000000180007198     ucrt:api-ms-win-crt-string-l1-1-0.dll
 0002:000001a0       \177api-ms-win-crt-string-l1-1-0_NULL_THUNK_DATA 00000001800071a0     ucrt:api-ms-win-crt-string-l1-1-0.dll
 0002:000001a8       __imp_JDK_Canonicalize     00000001800071a8     java:java.dll
 0002:000001b0       \177java_NULL_THUNK_DATA   00000001800071b0     java:java.dll
 0002:000001b8       __imp_JLI_ManifestIterate  00000001800071b8     jli:jli.dll
 0002:000001c0       \177jli_NULL_THUNK_DATA    00000001800071c0     jli:jli.dll
 0002:000001c8       __imp_JVM_PrintWarningAtDynamicAgentLoad 00000001800071c8     jvm:jvm.dll
 0002:000001d0       \177jvm_NULL_THUNK_DATA    00000001800071d0     jvm:jvm.dll
 0002:000001d8       __guard_check_icall_fptr   00000001800071d8     MSVCRT:guard_support.obj
 0002:000001e0       __guard_xfg_check_icall_fptr 00000001800071e0     MSVCRT:guard_support.obj
 0002:000001e8       __guard_dispatch_icall_fptr 00000001800071e8     MSVCRT:guard_support.obj
 0002:000001f0       __guard_xfg_dispatch_icall_fptr 00000001800071f0     MSVCRT:guard_support.obj
 0002:000001f8       __guard_xfg_table_dispatch_icall_fptr 00000001800071f8     MSVCRT:guard_support.obj
 0002:00000200       __castguard_check_failure_os_handled_fptr 0000000180007200     MSVCRT:guard_support.obj
 0002:00000208       __guard_memcpy_fptr        0000000180007208     vcruntime:softmemtag.obj
 0002:00000210       __xc_a                     0000000180007210     MSVCRT:initializers.obj
 0002:00000218       __xc_z                     0000000180007218     MSVCRT:initializers.obj
 0002:00000220       __xi_a                     0000000180007220     MSVCRT:initializers.obj
 0002:00000228       __xi_z                     0000000180007228     MSVCRT:initializers.obj
 0002:00000230       __xp_a                     0000000180007230     MSVCRT:initializers.obj
 0002:00000238       __xp_z                     0000000180007238     MSVCRT:initializers.obj
 0002:00000240       __xt_a                     0000000180007240     MSVCRT:initializers.obj
 0002:00000248       __xt_z                     0000000180007248     MSVCRT:initializers.obj
 0002:00000250       ??_C@_0CK@PECNJIMP@OOM?5error?5in?5native?5tmp?5buffer?5@ 0000000180007250     FileSystemSupport_md.obj
 0002:0000027c       ??_C@_04LOAJBDKD@true@     000000018000727c     InvocationAdapter.obj
 0002:00000288       ??_C@_0BF@MPBBPFEA@Can?9Redefine?9Classes@ 0000000180007288     InvocationAdapter.obj
 0002:000002a0       ??_C@_0BI@DOGNCBOD@Can?9Retransform?9Classes@ 00000001800072a0     InvocationAdapter.obj
 0002:000002b8       ??_C@_0BN@GGMNHHCI@Can?9Set?9Native?9Method?9Prefix@ 00000001800072b8     InvocationAdapter.obj
 0002:000002d8       ??_C@_0CD@ONCIGEJ@Can?9Maintain?9Original?9Method?9Or@ 00000001800072d8     InvocationAdapter.obj
 0002:00000300       ??_C@_0CI@HNHEPCMG@?9javaagent?3?5memory?5allocation?5f@ 0000000180007300     InvocationAdapter.obj
 0002:00000328       ??_C@_0DF@GEAEBGFM@Error?5opening?5zip?5file?5or?5JAR?5m@ 0000000180007328     InvocationAdapter.obj
 0002:00000360       ??_C@_0O@FJIJHIPN@Premain?9Class@ 0000000180007360     InvocationAdapter.obj
 0002:00000370       ??_C@_0DH@NNDEJOON@Failed?5to?5find?5Premain?9Class?5ma@ 0000000180007370     InvocationAdapter.obj
 0002:000003a8       ??_C@_0CM@BAFHELIF@?9javaagent?3?5Premain?9Class?5value@ 00000001800073a8     InvocationAdapter.obj
 0002:000003d8       ??_C@_0CG@MGGAPOHH@?9javaagent?3?5memory?5allocation?5f@ 00000001800073d8     InvocationAdapter.obj
 0002:00000400       ??_C@_0BA@EEOHCMMC@Boot?9Class?9Path@ 0000000180007400     InvocationAdapter.obj
 0002:00000410       ??_C@_0DO@FCLCEKPM@java?4lang?4instrument?1?9javaagent@ 0000000180007410     InvocationAdapter.obj
 0002:00000450       ??_C@_0EJ@MNINEPDM@java?4lang?4instrument?1?9javaagent@ 0000000180007450     InvocationAdapter.obj
 0002:000004a0       ??_C@_0DG@GEFLELM@java?4lang?4instrument?1?9javaagent@ 00000001800074a0     InvocationAdapter.obj
 0002:000004d8       ??_C@_0CI@DPANPEKD@?9javaagent?3?5agent?5class?5not?5spe@ 00000001800074d8     InvocationAdapter.obj
 0002:00000500       ??_C@_0DA@KPCNALNC@java?4lang?4instrument?1?9javaagent@ 0000000180007500     InvocationAdapter.obj
 0002:00000530       ??_C@_0EF@HEMJBLDG@s?2src?2java?4instrument?2share?2nat@ 0000000180007530     InvocationAdapter.obj
 0002:00000578       ??_C@_0P@CKGKOICP@result?$DN?$DNJNI_OK@ 0000000180007578     InvocationAdapter.obj
 0002:00000588       ??_C@_0DE@KGGELLFG@Error?5opening?5zip?5file?5or?5JAR?5m@ 0000000180007588     InvocationAdapter.obj
 0002:000005c0       ??_C@_0M@HHCNJNFE@Agent?9Class@ 00000001800075c0     InvocationAdapter.obj
 0002:000005d0       ??_C@_0DH@DADPHJGN@Failed?5to?5find?5Agent?9Class?5mani@ 00000001800075d0     InvocationAdapter.obj
 0002:00000610       ??_C@_0GG@HGIJBLPF@Unable?5to?5add?5?$CFs?5to?5system?5clas@ 0000000180007610     InvocationAdapter.obj
 0002:00000678       ??_C@_0BO@PHLNGFOC@Agent?9Class?5value?5is?5too?5big?6@ 0000000180007678     InvocationAdapter.obj
 0002:00000698       ??_C@_0CB@BKJLFFB@createInstrumentationImpl?5faile@ 0000000180007698     InvocationAdapter.obj
 0002:000006c0       ??_C@_07IPNMCAN@success@   00000001800076c0     InvocationAdapter.obj
 0002:000006c8       ??_C@_0CB@MDKECFOK@setLivePhaseEventHandlers?5faile@ 00000001800076c8     InvocationAdapter.obj
 0002:000006f0       ??_C@_0BG@PBIGODFM@startJavaAgent?5failed@ 00000001800076f0     InvocationAdapter.obj
 0002:00000708       ??_C@_0BI@FNNMMHD@Agent?5failed?5to?5start?$CB?6@ 0000000180007708     InvocationAdapter.obj
 0002:00000720       ??_C@_0BF@JIBAFKML@Launcher?9Agent?9Class@ 0000000180007720     InvocationAdapter.obj
 0002:00000738       ??_C@_0BL@ENCPOIKC@java?1lang?1OutOfMemoryError@ 0000000180007738     InvocationAdapter.obj
 0002:00000753       ??_C@_00CNPNBAHC@@         0000000180007753     InvocationAdapter.obj
 0002:00000760       ??_C@_0EC@FMFJIMAJ@processing?5of?5?9javaagent?5failed@ 0000000180007760     InvocationAdapter.obj
 0002:000007b0       ??_C@_0JF@EOMLGCNE@Unable?5to?5add?5?$CFs?5to?5system?5clas@ 00000001800077b0     InvocationAdapter.obj
 0002:00000850       ??_C@_0EH@PGNCMPLF@processing?5of?5?9javaagent?5failed@ 0000000180007850     InvocationAdapter.obj
 0002:00000898       ??_C@_0DJ@BIOAMFJP@processing?5of?5?9javaagent?5failed@ 0000000180007898     InvocationAdapter.obj
 0002:000008d4       ??_C@_01GBGANLPD@0@        00000001800078d4     InvocationAdapter.obj
 0002:000008e0       ??_C@_0FE@GJAPONAI@System?5class?5loader?5does?5not?5de@ 00000001800078e0     InvocationAdapter.obj
 0002:00000940       ??_C@_0EA@GNNEHPOG@Unexpected?5error?5?$CI?$CFd?$CJ?5returned?5@ 0000000180007940     InvocationAdapter.obj
 0002:00000980       ??_C@_0BE@JIIENKGJ@path?5?$CB?$DN?5?$CIchar?$CK?$CJNULL@ 0000000180007980     InvocationAdapter.obj
 0002:00000998       ??_C@_0DJ@KAMKBHCJ@WARNING?3?5illegal?5character?5in?5B@ 0000000180007998     InvocationAdapter.obj
 0002:000009d8       ??_C@_0BL@EGNHKKEM@?$CIvoid?$CK?$CJpath?5?$CB?$DN?5?$CIvoid?$CK?$CJNULL@ 00000001800079d8     InvocationAdapter.obj
 0002:000009f8       ??_C@_0CE@BMNGMKPL@WARNING?3?5unable?5to?5canonicalize@ 00000001800079f8     InvocationAdapter.obj
 0002:00000a20       ??_C@_0BG@LFGEPDCD@parent?5?$CB?$DN?5?$CIchar?$CK?$CJNULL@ 0000000180007a20     InvocationAdapter.obj
 0002:00000a38       ??_C@_0DJ@BINIAAK@WARNING?3?5?$CFs?5not?5added?5to?5bootst@ 0000000180007a38     InvocationAdapter.obj
 0002:00000a78       ??_C@_0CC@HMBHOALF@Illegal?5argument?5or?5not?5JAR?5fil@ 0000000180007a78     InvocationAdapter.obj
 0002:00000aa0       ??_C@_0BG@IPMFCDFJ@Unexpected?5error?3?5?$CFd?6@ 0000000180007aa0     InvocationAdapter.obj
 0002:00000ab8       ??_C@_0DO@NEGKBKCG@s?2src?2java?4instrument?2share?2nat@ 0000000180007ab8     JPLISAgent.obj
 0002:00000af8       ??_C@_0BP@JFPONFCF@jvmtierror?5?$DN?$DN?5JVMTI_ERROR_NONE@ 0000000180007af8     JPLISAgent.obj
 0002:00000b18       ??_C@_0BE@JEGDIMFH@environment?5?$CB?$DN?5NULL@ 0000000180007b18     JPLISAgent.obj
 0002:00000b30       ??_C@_0CD@EAGMGAOH@environment?9?$DOmJVMTIEnv?5?$DN?$DN?5jvmti@ 0000000180007b30     JPLISAgent.obj
 0002:00000b58       ??_C@_0BF@ENNAMHOI@fallback?5init?5failed@ 0000000180007b58     JPLISAgent.obj
 0002:00000b70       ??_C@_06KJFADLGN@result@   0000000180007b70     JPLISAgent.obj
 0002:00000b78       ??_C@_0CJ@MKNLGBML@instrumentation?5instance?5creati@ 0000000180007b78     JPLISAgent.obj
 0002:00000ba8       ??_C@_0CJ@BCMDJAKB@setting?5of?5live?5phase?5VM?5handle@ 0000000180007ba8     JPLISAgent.obj
 0002:00000bd8       ??_C@_0BP@DKNGPINN@agent?5load?1premain?5call?5failed@ 0000000180007bd8     JPLISAgent.obj
 0002:00000bf8       ??_C@_0CE@GJDJNDGE@commandStringIntoJavaStrings?5fa@ 0000000180007bf8     JPLISAgent.obj
 0002:00000c20       ??_C@_0CB@MHJJDMBL@invokeJavaAgentMainMethod?5faile@ 0000000180007c20     JPLISAgent.obj
 0002:00000c48       ??_C@_0CD@FJABNFOF@sun?1instrument?1InstrumentationI@ 0000000180007c48     JPLISAgent.obj
 0002:00000c70       ??_C@_0CJ@HOIGMIGF@find?5class?5on?5InstrumentationIm@ 0000000180007c70     JPLISAgent.obj
 0002:00000ca0       ??_C@_0BC@NFAEECCL@?$CBerrorOutstanding@ 0000000180007ca0     JPLISAgent.obj
 0002:00000cb8       ??_C@_07PAEOOHMC@?$CIJZZZ?$CJV@ 0000000180007cb8     JPLISAgent.obj
 0002:00000cc0       ??_C@_06FALKBLGB@?$DMinit?$DO@ 0000000180007cc0     JPLISAgent.obj
 0002:00000cc8       ??_C@_0CP@DNJEEBBF@find?5constructor?5on?5Instrumenta@ 0000000180007cc8     JPLISAgent.obj
 0002:00000cf8       ??_C@_0CP@HELLCCDH@call?5constructor?5on?5Instrumenta@ 0000000180007cf8     JPLISAgent.obj
 0002:00000d28       ??_C@_0BN@KICHEFJM@copy?5local?5ref?5to?5global?5ref@ 0000000180007d28     JPLISAgent.obj
 0002:00000d48       ??_C@_0CI@HEGLGDKJ@?$CILjava?1lang?1String?$DLLjava?1lang?1S@ 0000000180007d48     JPLISAgent.obj
 0002:00000d70       ??_C@_0BI@MHLLCGNO@loadClassAndCallPremain@ 0000000180007d70     JPLISAgent.obj
 0002:00000d88       ??_C@_0CE@KECKFJKE@can?8t?5find?5premain?5invoker?5meth@ 0000000180007d88     JPLISAgent.obj
 0002:00000db0       ??_C@_0BK@JAOFMOJK@loadClassAndCallAgentmain@ 0000000180007db0     JPLISAgent.obj
 0002:00000dd0       ??_C@_0CG@DOGNAPEF@can?8t?5find?5agentmain?5invoker?5me@ 0000000180007dd0     JPLISAgent.obj
 0002:00000e00       ??_C@_0HE@BEDHLJCA@?$CILjava?1lang?1Module?$DLLjava?1lang?1C@ 0000000180007e00     JPLISAgent.obj
 0002:00000e78       ??_C@_09IFONHNKG@transform@ 0000000180007e78     JPLISAgent.obj
 0002:00000e88       ??_C@_0BO@LKBEMJID@can?8t?5find?5transform?5methodID@ 0000000180007e88     JPLISAgent.obj
 0002:00000ea8       ??_C@_0CE@NNNMFAHP@can?8t?5create?5class?5name?5java?5st@ 0000000180007ea8     JPLISAgent.obj
 0002:00000ed0       ??_C@_0CB@GCBHBCEC@can?8t?5create?5options?5java?5strin@ 0000000180007ed0     JPLISAgent.obj
 0002:00000ef8       ??_C@_0BK@OLJIPBJG@mainCallingMethod?5?$CB?$DN?5NULL@ 0000000180007ef8     JPLISAgent.obj
 0002:00000f20       ??_C@_0ED@CEAHFGIB@Outstanding?5error?5when?5calling?5@ 0000000180007f20     JPLISAgent.obj
 0002:00000f70       ??_C@_0EK@NBNNLAGF@jvmtierror?5?$DN?$DN?5JVMTI_ERROR_NONE?5@ 0000000180007f70     JPLISAgent.obj
 0002:00000fc0       ??_C@_0CC@NONNBMCM@error?5in?5the?5JVMTI?5GetNamedModu@ 0000000180007fc0     JPLISAgent.obj
 0002:00000fe8       ??_C@_0BI@GCGOKABC@err?5?$DN?$DN?5JVMTI_ERROR_NONE@ 0000000180007fe8     JPLISAgent.obj
 0002:00001000       ??_C@_0BJ@OFPEOMG@can?8t?5create?5name?5string@ 0000000180008000     JPLISAgent.obj
 0002:00001020       ??_C@_0BI@KDNOCEBM@can?8t?5create?5byte?5array@ 0000000180008020     JPLISAgent.obj
 0002:00001038       ??_C@_0BM@NODFBCMB@can?8t?5set?5byte?5array?5region@ 0000000180008038     JPLISAgent.obj
 0002:00001058       ??_C@_0CE@NCFBINFF@agent?9?$DOmInstrumentationImpl?5?$CB?$DN?5@ 0000000180008058     JPLISAgent.obj
 0002:00001080       ??_C@_0BK@GEFGBHIE@agent?9?$DOmTransform?5?$CB?$DN?5NULL@ 0000000180008080     JPLISAgent.obj
 0002:000010a0       ??_C@_0BN@JDJGIEH@transform?5method?5call?5failed@ 00000001800080a0     JPLISAgent.obj
 0002:000010c0       ??_C@_0BH@DDPAAIBF@can?8t?5get?5array?5length@ 00000001800080c0     JPLISAgent.obj
 0002:000010d8       ??_C@_0BN@KNPJDEBO@can?8t?5allocate?5result?5buffer@ 00000001800080d8     JPLISAgent.obj
 0002:000010f8       ??_C@_0BM@CLGDMLIA@can?8t?5get?5byte?5array?5region@ 00000001800080f8     JPLISAgent.obj
 0002:00001118       ??_C@_0BK@JCFBFKNG@isSafeForJNICalls?$CIjnienv?$CJ@ 0000000180008118     JPLISAgent.obj
 0002:00001138       ??_C@_0CF@PBJJFPHF@?$CBisUnchecked?$CIjnienv?0?5throwableT@ 0000000180008138     JPLISAgent.obj
 0002:00001160       ??_C@_0CB@KCPANAMN@java?1lang?1ClassNotFoundExceptio@ 0000000180008160     JPLISAgent.obj
 0002:00001188       ??_C@_0DA@MJOAEAPC@java?1lang?1instrument?1Unmodifiab@ 0000000180008188     JPLISAgent.obj
 0002:000011b8       ??_C@_0BA@JJLOPNCP@java?1lang?1Class@ 00000001800081b8     JPLISAgent.obj
 0002:000011c8       ??_C@_0BO@GBLMHFAI@FindClass?5returned?5null?5class@ 00000001800081c8     JPLISAgent.obj
 0002:000011e8       ??_C@_0BI@JLMJJPLE@classArrayClass?5?$CB?$DN?5NULL@ 00000001800081e8     JPLISAgent.obj
 0002:00001200       ??_C@_0CD@NMCFBNHK@NewObjectArray?5returned?5null?5ar@ 0000000180008200     JPLISAgent.obj
 0002:00001228       ??_C@_0BD@BNJLEHDL@localArray?5?$CB?$DN?5NULL@ 0000000180008228     JPLISAgent.obj
 0002:00001240       ??_C@_0CI@MJAJKCDF@jvmtierror?5?$DN?$DN?5JVMTI_ERROR_NOT_A@ 0000000180008240     JPLISAgent.obj
 0002:00001268       ??_C@_0BB@DBNGJIMM@jvmtienv?5?$CB?$DN?5NULL@ 0000000180008268     JPLISAgent.obj
 0002:00001280       ??_C@_0BJ@EJCHPAPK@retransformerEnv?5?$CB?$DN?5NULL@ 0000000180008280     JPLISAgent.obj
 0002:000012a0       ??_C@_0BA@DKKKAEPC@classes?5?$CB?$DN?5NULL@ 00000001800082a0     JPLISAgent.obj
 0002:000012b0       ??_C@_0P@IBHCMEIB@?$CBerrorOccurred@ 00000001800082b0     JPLISAgent.obj
 0002:000012c0       ??_C@_0BA@DHKCDHMI@numClasses?5?$CB?$DN?50@ 00000001800082c0     JPLISAgent.obj
 0002:000012d0       ??_C@_0BK@HBLAKIEB@classArray?$FLindex?$FN?5?$CB?$DN?5NULL@ 00000001800082d0     JPLISAgent.obj
 0002:000012f0       ??_C@_0BJ@NGKAGHPG@classDefinitions?5?$CB?$DN?5NULL@ 00000001800082f0     JPLISAgent.obj
 0002:00001310       ??_C@_0M@KGLONNBG@numDefs?5?$DO?50@ 0000000180008310     JPLISAgent.obj
 0002:00001320       ??_C@_0CF@BGAIILOJ@java?1lang?1instrument?1ClassDefin@ 0000000180008320     JPLISAgent.obj
 0002:00001348       ??_C@_0BE@IIFEGCLG@?$CI?$CJLjava?1lang?1Class?$DL@ 0000000180008348     JPLISAgent.obj
 0002:00001360       ??_C@_0BD@FFKMDMBN@getDefinitionClass@ 0000000180008360     JPLISAgent.obj
 0002:00001374       ??_C@_04LHPAGAEF@?$CI?$CJ?$FLB@ 0000000180008374     JPLISAgent.obj
 0002:00001380       ??_C@_0BH@FOGLHNOO@getDefinitionClassFile@ 0000000180008380     JPLISAgent.obj
 0002:00001398       ??_C@_0BE@NLJNCPBN@prefixArray?5?$CB?$DN?5NULL@ 0000000180008398     JPLISAgent.obj
 0002:000013b0       ??_C@_0EE@FPMMKFJK@?$CK?$CK?$CK?5java?4lang?4instrument?5ASSERT@ 00000001800083b0     JPLISAssert.obj
 0002:00001400       ??_C@_0FE@HCMNEDKA@?$CK?$CK?$CK?5java?4lang?4instrument?5ASSERT@ 0000000180008400     JPLISAssert.obj
 0002:00001460       ??_C@_0EC@BMPNKMFA@s?2src?2java?4instrument?2share?2nat@ 0000000180008460     JavaExceptions.obj
 0002:000014a8       ??_C@_0BH@EKGMOCH@throwableToMap?5?$CB?$DN?5NULL@ 00000001800084a8     JavaExceptions.obj
 0002:000014c0       ??_C@_0BC@HKCJMFCP@className?5?$CB?$DN?5NULL@ 00000001800084c0     JavaExceptions.obj
 0002:000014d8       ??_C@_0BG@IKDDPPGD@?$CILjava?1lang?1String?$DL?$CJV@ 00000001800084d8     JavaExceptions.obj
 0002:000014f0       ??_C@_0BI@NBLNIHIB@java?1lang?1InternalError@ 00000001800084f0     JavaExceptions.obj
 0002:00001508       ??_C@_0BP@GJLHLAKJ@java?1lang?1NullPointerException@ 0000000180008508     JavaExceptions.obj
 0002:00001528       ??_C@_0CD@MOHADDFA@java?1lang?1IllegalArgumentExcept@ 0000000180008528     JavaExceptions.obj
 0002:00001550       ??_C@_0CA@OCDKFHGJ@java?1lang?1ClassCircularityError@ 0000000180008550     JavaExceptions.obj
 0002:00001570       ??_C@_0BG@FNCILCAN@java?1lang?1VerifyError@ 0000000180008570     JavaExceptions.obj
 0002:00001588       ??_C@_0CI@LDDEGNGM@java?1lang?1UnsupportedOperationE@ 0000000180008588     JavaExceptions.obj
 0002:000015b0       ??_C@_0DF@IFGMNJBO@class?5redefinition?5failed?3?5atte@ 00000001800085b0     JavaExceptions.obj
 0002:000015f0       ??_C@_0EO@LOHFEPOO@class?5redefinition?5failed?3?5atte@ 00000001800085f0     JavaExceptions.obj
 0002:00001640       ??_C@_0EI@PJGIIEAK@class?5redefinition?5failed?3?5atte@ 0000000180008640     JavaExceptions.obj
 0002:00001688       ??_C@_0DI@KJLEIONK@class?5redefinition?5failed?3?5atte@ 0000000180008688     JavaExceptions.obj
 0002:000016c0       ??_C@_0ED@PPHPPFFE@class?5redefinition?5failed?3?5atte@ 00000001800086c0     JavaExceptions.obj
 0002:00001710       ??_C@_0HJ@FGKDIDEP@class?5redefinition?5failed?3?5atte@ 0000000180008710     JavaExceptions.obj
 0002:00001790       ??_C@_0EA@INKOHMMN@class?5redefinition?5failed?3?5atte@ 0000000180008790     JavaExceptions.obj
 0002:000017d0       ??_C@_0CH@DNCLOIOF@java?1lang?1UnsupportedClassVersi@ 00000001800087d0     JavaExceptions.obj
 0002:000017f8       ??_C@_0BP@NAHGIHIH@java?1lang?1NoClassDefFoundError@ 00000001800087f8     JavaExceptions.obj
 0002:00001818       ??_C@_0BI@MAPDCENK@class?5names?5don?8t?5match@ 0000000180008818     JavaExceptions.obj
 0002:00001830       ??_C@_0BL@EEAIAIEG@java?1lang?1ClassFormatError@ 0000000180008830     JavaExceptions.obj
 0002:00001850       ??_C@_0CJ@DNCKJBBE@class?5redefinition?5failed?3?5inva@ 0000000180008850     JavaExceptions.obj
 0002:00001880       ??_C@_0BG@JKFIFBMN@unsupported?5operation@ 0000000180008880     JavaExceptions.obj
 0002:00001898       ??_C@_0CD@LAOKENHO@can?8t?5create?5exception?5java?5str@ 0000000180008898     JavaExceptions.obj
 0002:000018c0       ??_C@_0BF@FOHFOJOB@?$CI?$CJLjava?1lang?1String?$DL@ 00000001800088c0     JavaExceptions.obj
 0002:000018d8       ??_C@_08JCDFGHAO@toString@ 00000001800088d8     JavaExceptions.obj
 0002:000018e8       ??_C@_0BA@NOLMKEPF@java?1lang?1Error@ 00000001800088e8     JavaExceptions.obj
 0002:000018f8       ??_C@_0BL@IONOAEOO@java?1lang?1RuntimeException@ 00000001800088f8     JavaExceptions.obj
 0002:00001918       ??_C@_0CC@GKBBLNKJ@throwThrowable?5failed?5to?5re?9thr@ 0000000180008918     JavaExceptions.obj
 0002:00001940       ??_C@_0BB@EJBOEPOM@result?5?$DN?$DN?5JNI_OK@ 0000000180008940     JavaExceptions.obj
 0002:00001958       ??_C@_09HLKPJHCC@?9_?4?$CB?$HO?$CK?8?$CI?$CJ@ 0000000180008958     PathCharsValidator.obj
 0002:00001968       ??_C@_07DDNJCNOL@?3?$EA?$CG?$DN?$CL$?0@ 0000000180008968     PathCharsValidator.obj
 0002:00001970       ??_C@_02DKJMBEPB@?$DL?1@   0000000180008970     PathCharsValidator.obj
 0002:00001978       ??_C@_0DO@IILOFBP@s?2src?2java?4instrument?2share?2nat@ 0000000180008978     Reentrancy.obj
 0002:000019b8       ??_C@_0BK@PPCACBKK@error?5?$DN?$DN?5JVMTI_ERROR_NONE@ 00000001800089b8     Reentrancy.obj
 0002:000019d8       ??_C@_0BB@LLFPNPAC@test?5?$DN?$DN?5expected@ 00000001800089d8     Reentrancy.obj
 0002:000019f0       ??_C@_0DN@HOJJMEHN@s?2src?2java?4instrument?2share?2nat@ 00000001800089f0     Utilities.obj
 0002:00001a30       ??_C@_0BI@NNKHJJFO@Can?8t?5deallocate?5memory@ 0000000180008a30     Utilities.obj
 0002:00001a48       _pDefaultRawDllMain        0000000180008a48     MSVCRT:dll_dllmain.obj
 0002:00001a48       _pRawDllMain               0000000180008a48     MSVCRT:dll_dllmain.obj
 0002:00001a60       __xmm@ffffffffffffffffffffffffffffffff 0000000180008a60     MSVCRT:utility.obj
 0002:00001a70       _load_config_used          0000000180008a70     MSVCRT:loadcfg.obj
 0002:00001c80       __volatile_metadata        0000000180008c80     <linker-defined>
 0002:00001fa8       __rtc_iaa                  0000000180008fa8     MSVCRT:initsect.obj
 0002:00001fb0       __rtc_izz                  0000000180008fb0     MSVCRT:initsect.obj
 0002:00001fb8       __rtc_taa                  0000000180008fb8     MSVCRT:initsect.obj
 0002:00001fc0       __rtc_tzz                  0000000180008fc0     MSVCRT:initsect.obj
 0002:000028c8       __IMPORT_DESCRIPTOR_java   00000001800098c8     java:java.dll
 0002:000028dc       __IMPORT_DESCRIPTOR_jli    00000001800098dc     jli:jli.dll
 0002:000028f0       __IMPORT_DESCRIPTOR_jvm    00000001800098f0     jvm:jvm.dll
 0002:00002904       __IMPORT_DESCRIPTOR_KERNEL32 0000000180009904     kernel32:KERNEL32.dll
 0002:00002918       __IMPORT_DESCRIPTOR_VCRUNTIME140 0000000180009918     vcruntime:VCRUNTIME140.dll
 0002:0000292c       __IMPORT_DESCRIPTOR_api-ms-win-crt-heap-l1-1-0 000000018000992c     ucrt:api-ms-win-crt-heap-l1-1-0.dll
 0002:00002940       __IMPORT_DESCRIPTOR_api-ms-win-crt-convert-l1-1-0 0000000180009940     ucrt:api-ms-win-crt-convert-l1-1-0.dll
 0002:00002954       __IMPORT_DESCRIPTOR_api-ms-win-crt-stdio-l1-1-0 0000000180009954     ucrt:api-ms-win-crt-stdio-l1-1-0.dll
 0002:00002968       __IMPORT_DESCRIPTOR_api-ms-win-crt-string-l1-1-0 0000000180009968     ucrt:api-ms-win-crt-string-l1-1-0.dll
 0002:0000297c       __IMPORT_DESCRIPTOR_api-ms-win-crt-runtime-l1-1-0 000000018000997c     ucrt:api-ms-win-crt-runtime-l1-1-0.dll
 0002:00002990       __NULL_IMPORT_DESCRIPTOR   0000000180009990     java:java.dll
 0003:00000000       __security_cookie_complement 000000018000b000     MSVCRT:gs_cookie.obj
 0003:00000008       __security_cookie          000000018000b008     MSVCRT:gs_cookie.obj
 0003:00000010       __scrt_native_dllmain_reason 000000018000b010     MSVCRT:utility.obj
 0003:00000018       __isa_available            000000018000b018     MSVCRT:cpu_disp.obj
 0003:0000001c       __isa_enabled              000000018000b01c     MSVCRT:cpu_disp.obj
 0003:00000020       __memset_fast_string_threshold 000000018000b020     MSVCRT:cpu_disp.obj
 0003:00000028       __memset_nt_threshold      000000018000b028     MSVCRT:cpu_disp.obj
 0003:00000030       __scrt_ucrt_dll_is_in_use  000000018000b030     MSVCRT:ucrt_stubs.obj
 0003:000005e0       ?__type_info_root_node@@3U__type_info_node@@A 000000018000b5e0     MSVCRT:tncleanup.obj
 0003:000005f0       ?_OptionsStorage@?1??__local_stdio_scanf_options@@9@4_KA 000000018000b5f0     MSVCRT:default_local_stdio_options.obj
 0003:000005f8       __scrt_current_native_startup_state 000000018000b5f8     MSVCRT:utility.obj
 0003:00000600       __scrt_native_startup_lock 000000018000b600     MSVCRT:utility.obj
 0003:00000640       __scrt_debugger_hook_flag  000000018000b640     MSVCRT:utility_desktop.obj
 0003:00000644       __favor                    000000018000b644     MSVCRT:cpu_disp.obj
 0003:00000648       ?_OptionsStorage@?1??__local_stdio_printf_options@@9@9 000000018000b648     <common>
 0003:00000650       __dyn_tls_init_callback    000000018000b650     <common>

 entry point at        0001:000053c0

 Static symbols

 0000:ffff1000       .debug$S                   0000000180000000     instrument.exp
 0000:ffff1000       .debug$S                   0000000180000000     vcruntime:VCRUNTIME140.dll
 0000:ffff1000       .debug$S                   0000000180000000     vcruntime:VCRUNTIME140.dll
 0000:ffff1000       .debug$S                   0000000180000000     vcruntime:VCRUNTIME140.dll
 0000:ffff1000       .debug$S                   0000000180000000     vcruntime:VCRUNTIME140.dll
 0000:ffff1000       .debug$S                   0000000180000000     vcruntime:VCRUNTIME140.dll
 0000:ffff1000       .debug$S                   0000000180000000     vcruntime:VCRUNTIME140.dll
 0000:ffff1000       .debug$S                   0000000180000000     vcruntime:VCRUNTIME140.dll
 0000:ffff1000       .debug$S                   0000000180000000     vcruntime:VCRUNTIME140.dll
 0000:ffff1000       .debug$S                   0000000180000000     ucrt:api-ms-win-crt-convert-l1-1-0.dll
 0000:ffff1000       .debug$S                   0000000180000000     ucrt:api-ms-win-crt-heap-l1-1-0.dll
 0000:ffff1000       .debug$S                   0000000180000000     ucrt:api-ms-win-crt-heap-l1-1-0.dll
 0000:ffff1000       .debug$S                   0000000180000000     ucrt:api-ms-win-crt-heap-l1-1-0.dll
 0000:ffff1000       .debug$S                   0000000180000000     ucrt:api-ms-win-crt-heap-l1-1-0.dll
 0000:ffff1000       .debug$S                   0000000180000000     ucrt:api-ms-win-crt-runtime-l1-1-0.dll
 0000:ffff1000       .debug$S                   0000000180000000     ucrt:api-ms-win-crt-runtime-l1-1-0.dll
 0000:ffff1000       .debug$S                   0000000180000000     ucrt:api-ms-win-crt-runtime-l1-1-0.dll
 0000:ffff1000       .debug$S                   0000000180000000     ucrt:api-ms-win-crt-runtime-l1-1-0.dll
 0000:ffff1000       .debug$S                   0000000180000000     ucrt:api-ms-win-crt-runtime-l1-1-0.dll
 0000:ffff1000       .debug$S                   0000000180000000     ucrt:api-ms-win-crt-runtime-l1-1-0.dll
 0000:ffff1000       .debug$S                   0000000180000000     ucrt:api-ms-win-crt-runtime-l1-1-0.dll
 0000:ffff1000       .debug$S                   0000000180000000     ucrt:api-ms-win-crt-runtime-l1-1-0.dll
 0000:ffff1000       .debug$S                   0000000180000000     ucrt:api-ms-win-crt-runtime-l1-1-0.dll
 0000:ffff1000       .debug$S                   0000000180000000     ucrt:api-ms-win-crt-runtime-l1-1-0.dll
 0000:ffff1000       .debug$S                   0000000180000000     ucrt:api-ms-win-crt-runtime-l1-1-0.dll
 0000:ffff1000       .debug$S                   0000000180000000     ucrt:api-ms-win-crt-runtime-l1-1-0.dll
 0000:ffff1000       .debug$S                   0000000180000000     ucrt:api-ms-win-crt-stdio-l1-1-0.dll
 0000:ffff1000       .debug$S                   0000000180000000     ucrt:api-ms-win-crt-stdio-l1-1-0.dll
 0000:ffff1000       .debug$S                   0000000180000000     ucrt:api-ms-win-crt-string-l1-1-0.dll
 0000:ffff1000       .debug$S                   0000000180000000     ucrt:api-ms-win-crt-string-l1-1-0.dll
 0000:ffff1000       .debug$S                   0000000180000000     ucrt:api-ms-win-crt-string-l1-1-0.dll
 0000:ffff1000       .debug$S                   0000000180000000     ucrt:api-ms-win-crt-string-l1-1-0.dll
 0000:ffff1000       .debug$S                   0000000180000000     ucrt:api-ms-win-crt-string-l1-1-0.dll
 0000:ffff1000       .debug$S                   0000000180000000     kernel32:KERNEL32.dll
 0000:ffff1000       .debug$S                   0000000180000000     kernel32:KERNEL32.dll
 0000:ffff1000       .debug$S                   0000000180000000     kernel32:KERNEL32.dll
 0000:ffff1000       .debug$S                   0000000180000000     kernel32:KERNEL32.dll
 0000:ffff1000       .debug$S                   0000000180000000     kernel32:KERNEL32.dll
 0000:ffff1000       .debug$S                   0000000180000000     kernel32:KERNEL32.dll
 0000:ffff1000       .debug$S                   0000000180000000     kernel32:KERNEL32.dll
 0000:ffff1000       .debug$S                   0000000180000000     kernel32:KERNEL32.dll
 0000:ffff1000       .debug$S                   0000000180000000     kernel32:KERNEL32.dll
 0000:ffff1000       .debug$S                   0000000180000000     kernel32:KERNEL32.dll
 0000:ffff1000       .debug$S                   0000000180000000     kernel32:KERNEL32.dll
 0000:ffff1000       .debug$S                   0000000180000000     kernel32:KERNEL32.dll
 0000:ffff1000       .debug$S                   0000000180000000     kernel32:KERNEL32.dll
 0000:ffff1000       .debug$S                   0000000180000000     kernel32:KERNEL32.dll
 0000:ffff1000       .debug$S                   0000000180000000     kernel32:KERNEL32.dll
 0000:ffff1000       .debug$S                   0000000180000000     kernel32:KERNEL32.dll
 0000:ffff1000       .debug$S                   0000000180000000     kernel32:KERNEL32.dll
 0000:ffff1000       .debug$S                   0000000180000000     kernel32:KERNEL32.dll
 0000:ffff1000       .debug$S                   0000000180000000     kernel32:KERNEL32.dll
 0000:ffff1000       .debug$S                   0000000180000000     kernel32:KERNEL32.dll
 0000:ffff1000       .debug$S                   0000000180000000     kernel32:KERNEL32.dll
 0000:ffff1000       .debug$S                   0000000180000000     kernel32:KERNEL32.dll
 0000:ffff1000       .debug$S                   0000000180000000     jvm:jvm.dll
 0000:ffff1000       .debug$S                   0000000180000000     java:java.dll
 0000:ffff1000       .debug$S                   0000000180000000     jli:jli.dll
 0001:000005b4       normalizePath              00000001800015b4 f   FileSystemSupport_md.obj
 0001:00001088       appendBootClassPath        0000000180002088 f   InvocationAdapter.obj
 0001:0000154c       appendClassPath            000000018000254c f   InvocationAdapter.obj
 0001:000019f0       parseArgumentTail          00000001800029f0 f   InvocationAdapter.obj
 0001:00002558       getModuleObject            0000000180003558 f   JPLISAgent.obj
 0001:00003f50       doAttribute                0000000180004f50 f   JarFacade.obj
 0001:0000498c       highMask                   000000018000598c f   PathCharsValidator.obj
 0001:000049cc       highMaskRange              00000001800059cc f   PathCharsValidator.obj
 0001:00004a28       initialize                 0000000180005a28 f   PathCharsValidator.obj
 0001:00004b24       lowMask                    0000000180005b24 f   PathCharsValidator.obj
 0001:00005070       $$000000                   0000000180006070     MSVCRT:amdsecgs.obj
 0001:000050a0       ?dllmain_crt_dispatch@@YAHQEAUHINSTANCE__@@KQEAX@Z 00000001800060a0 f   MSVCRT:dll_dllmain.obj
 0001:000050f0       ?dllmain_crt_process_attach@@YAHQEAUHINSTANCE__@@QEAX@Z 00000001800060f0 f   MSVCRT:dll_dllmain.obj
 0001:00005208       ?dllmain_crt_process_detach@@YAH_N@Z 0000000180006208 f   MSVCRT:dll_dllmain.obj
 0001:0000528c       ?dllmain_dispatch@@YAHQEAUHINSTANCE__@@KQEAX@Z 000000018000628c f   MSVCRT:dll_dllmain.obj
 0001:00005508       capture_previous_context   0000000180006508 f   MSVCRT:gs_report.obj
 0001:00005dc0       $$000000                   0000000180006dc0     MSVCRT:guard_dispatch.obj
 0001:00005de0       $$000000                   0000000180006de0     MSVCRT:guard_xfg_dispatch.obj
 0001:00005df6       ?fin$0@?0??dllmain_crt_process_attach@@YAHQEAUHINSTANCE__@@QEAX@Z@4HA 0000000180006df6 f   MSVCRT:dll_dllmain.obj
 0001:00005e0d       ?fin$0@?0??dllmain_crt_process_detach@@YAH_N@Z@4HA 0000000180006e0d f   MSVCRT:dll_dllmain.obj
 0001:00005e26       ?fin$1@?0??dllmain_crt_process_detach@@YAH_N@Z@4HA 0000000180006e26 f   MSVCRT:dll_dllmain.obj
 0001:00005e3a       ?filt$0@?0??dllmain_dispatch@@YAHQEAUHINSTANCE__@@KQEAX@Z@4HA 0000000180006e3a f   MSVCRT:dll_dllmain.obj
 0001:00005e70       __scrt_is_nonwritable_in_current_image$filt$0 0000000180006e70 f   MSVCRT:utility.obj
 0002:00001a50       GS_ExceptionPointers       0000000180008a50     MSVCRT:gs_report.obj
 0002:00001fc8       $unwind$modifiedUtf8LengthOfUtf8 0000000180008fc8     EncodingSupport.obj
 0002:00001fd0       $unwind$convertUtf8ToModifiedUtf8 0000000180008fd0     EncodingSupport.obj
 0002:00001fe4       $unwind$convertUtf8ToPlatformString 0000000180008fe4     EncodingSupport_md.obj
 0002:00002004       $unwind$fprintf            0000000180009004     FileSystemSupport_md.obj
 0002:00002010       $unwind$basePath           0000000180009010     FileSystemSupport_md.obj
 0002:00002010       $unwind$doAttribute        0000000180009010     JarFacade.obj
 0002:00002024       $unwind$normalizePath      0000000180009024     FileSystemSupport_md.obj
 0002:0000203c       $unwind$isAbsolute         000000018000903c     FileSystemSupport_md.obj
 0002:0000203c       $unwind$normalize_path     000000018000903c     FileSystemSupport_md.obj
 0002:0000203c       $unwind$Java_sun_instrument_InstrumentationImpl_loadAgent0 000000018000903c     InstrumentationImplNativeMethods.obj
 0002:0000203c       $unwind$appendClassPath    000000018000903c     InvocationAdapter.obj
 0002:0000203c       $unwind$getBooleanAttribute 000000018000903c     InvocationAdapter.obj
 0002:0000203c       $unwind$addNativeMethodPrefixCapability 000000018000903c     JPLISAgent.obj
 0002:0000203c       $unwind$deallocateCommandLineData 000000018000903c     JPLISAgent.obj
 0002:0000203c       $unwind$createAndThrowInternalError 000000018000903c     JavaExceptions.obj
 0002:0000203c       $unwind$createAndThrowThrowableFromJVMTIErrorCode 000000018000903c     JavaExceptions.obj
 0002:0000203c       $unwind$initializeFallbackError 000000018000903c     JavaExceptions.obj
 0002:0000203c       $unwind$logThrowable       000000018000903c     JavaExceptions.obj
 0002:0000203c       $unwind$highMask           000000018000903c     PathCharsValidator.obj
 0002:0000203c       $unwind$lowMask            000000018000903c     PathCharsValidator.obj
 0002:0000203c       $unwind$assertTLSValue     000000018000903c     Reentrancy.obj
 0002:0000203c       $unwind$__raise_securityfailure 000000018000903c     MSVCRT:gs_report.obj
 0002:0000203c       $unwind$__scrt_initialize_crt 000000018000903c     MSVCRT:utility.obj
 0002:0000203c       $unwind$__scrt_initialize_onexit_tables 000000018000903c     MSVCRT:utility.obj
 0002:0000203c       $unwind$__scrt_release_startup_lock 000000018000903c     MSVCRT:utility.obj
 0002:0000203c       $unwind$__scrt_uninitialize_crt 000000018000903c     MSVCRT:utility.obj
 0002:00002044       $unwind$resolve            0000000180009044     FileSystemSupport_md.obj
 0002:00002060       $unwind$fromURIPath        0000000180009060     FileSystemSupport_md.obj
 0002:00002060       $unwind$eventHandlerVMInit 0000000180009060     InvocationAdapter.obj
 0002:00002060       $unwind$confirmingTLSSet   0000000180009060     Reentrancy.obj
 0002:00002060       $unwind$__scrt_dllmain_exception_filter 0000000180009060     MSVCRT:utility.obj
 0002:00002074       $unwind$Agent_OnLoad       0000000180009074     InvocationAdapter.obj
 0002:0000208c       $unwind$Agent_OnAttach     000000018000908c     InvocationAdapter.obj
 0002:000020a4       $unwind$eventHandlerClassFileLoadHook 00000001800090a4     InvocationAdapter.obj
 0002:000020bc       $unwind$appendBootClassPath 00000001800090bc     InvocationAdapter.obj
 0002:000020e0       $unwind$parseArgumentTail  00000001800090e0     InvocationAdapter.obj
 0002:000020e0       $unwind$recordCommandLineData 00000001800090e0     JPLISAgent.obj
 0002:000020e0       $unwind$getMessageFromThrowable 00000001800090e0     JavaExceptions.obj
 0002:000020f8       $unwind$convertCapabilityAttributes 00000001800090f8     InvocationAdapter.obj
 0002:000020f8       $unwind$getObjectSize      00000001800090f8     JPLISAgent.obj
 0002:000020f8       $unwind$redefineClassMapper 00000001800090f8     JPLISAgent.obj
 0002:000020f8       $unwind$setHasRetransformableTransformers 00000001800090f8     JPLISAgent.obj
 0002:000020f8       $unwind$setHasTransformers 00000001800090f8     JPLISAgent.obj
 0002:000020f8       $unwind$getAttribute       00000001800090f8     JarFacade.obj
 0002:000020f8       $unwind$checkForAndClearThrowable 00000001800090f8     JavaExceptions.obj
 0002:000020f8       $unwind$isUnchecked        00000001800090f8     JavaExceptions.obj
 0002:000020f8       $unwind$mapAllCheckedToInternalErrorMapper 00000001800090f8     JavaExceptions.obj
 0002:000020f8       $unwind$preserveThrowable  00000001800090f8     JavaExceptions.obj
 0002:000020f8       $unwind$releaseReentrancyToken 00000001800090f8     Reentrancy.obj
 0002:000020f8       $unwind$_RTC_Initialize    00000001800090f8     MSVCRT:initsect.obj
 0002:000020f8       $unwind$_RTC_Terminate     00000001800090f8     MSVCRT:initsect.obj
 0002:00002104       $unwind$loadAgent          0000000180009104     InvocationAdapter.obj
 0002:0000211c       $unwind$getJPLISEnvironment 000000018000911c     JPLISAgent.obj
 0002:0000212c       $unwind$createNewJPLISAgent 000000018000912c     JPLISAgent.obj
 0002:00002140       $unwind$addRedefineClassesCapability 0000000180009140     JPLISAgent.obj
 0002:00002140       $unwind$checkCapabilities  0000000180009140     JPLISAgent.obj
 0002:00002154       $unwind$addOriginalMethodOrderCapability 0000000180009154     JPLISAgent.obj
 0002:00002154       $unwind$enableNativeMethodPrefixCapability 0000000180009154     JPLISAgent.obj
 0002:00002164       $unwind$createInstrumentationImpl 0000000180009164     JPLISAgent.obj
 0002:00002180       $unwind$setLivePhaseEventHandlers 0000000180009180     JPLISAgent.obj
 0002:00002190       $unwind$startJavaAgent     0000000180009190     JPLISAgent.obj
 0002:000021a0       $unwind$processJavaStart   00000001800091a0     JPLISAgent.obj
 0002:000021a0       $unwind$createThrowableFromJVMTIErrorCode 00000001800091a0     JavaExceptions.obj
 0002:000021b0       $unwind$transformClassFile 00000001800091b0     JPLISAgent.obj
 0002:000021cc       $unwind$retransformableEnvironment 00000001800091cc     JPLISAgent.obj
 0002:000021ec       $unwind$isModifiableClass  00000001800091ec     JPLISAgent.obj
 0002:000021ec       $unwind$isSafeForJNICalls  00000001800091ec     JavaExceptions.obj
 0002:000021ec       $unwind$__scrt_initialize_default_local_stdio_options 00000001800091ec     MSVCRT:default_local_stdio_options.obj
 0002:000021ec       $unwind$?dllmain_crt_dispatch@@YAHQEAUHINSTANCE__@@KQEAX@Z 00000001800091ec     MSVCRT:dll_dllmain.obj
 0002:000021ec       $unwind$DllMain            00000001800091ec     MSVCRT:dll_dllmain_stub.obj
 0002:000021ec       $unwind$__GSHandlerCheck   00000001800091ec     MSVCRT:gshandler.obj
 0002:000021ec       $unwind$__scrt_acquire_startup_lock 00000001800091ec     MSVCRT:utility.obj
 0002:000021ec       $unwind$__scrt_dllmain_after_initialize_c 00000001800091ec     MSVCRT:utility.obj
 0002:000021ec       $unwind$__scrt_dllmain_before_initialize_c 00000001800091ec     MSVCRT:utility.obj
 0002:000021ec       $unwind$__scrt_dllmain_crt_thread_attach 00000001800091ec     MSVCRT:utility.obj
 0002:000021ec       $unwind$__scrt_dllmain_crt_thread_detach 00000001800091ec     MSVCRT:utility.obj
 0002:000021ec       $unwind$__scrt_dllmain_uninitialize_c 00000001800091ec     MSVCRT:utility.obj
 0002:000021ec       $unwind$__scrt_dllmain_uninitialize_critical 00000001800091ec     MSVCRT:utility.obj
 0002:000021f4       $unwind$retransformClasses 00000001800091f4     JPLISAgent.obj
 0002:0000220c       $unwind$redefineClasses    000000018000920c     JPLISAgent.obj
 0002:00002224       $unwind$appendToClassLoaderSearch 0000000180009224     JPLISAgent.obj
 0002:00002244       $unwind$setNativeMethodPrefixes 0000000180009244     JPLISAgent.obj
 0002:0000225c       $unwind$initializeJPLISAgent 000000018000925c     JPLISAgent.obj
 0002:00002270       $unwind$commandStringIntoJavaStrings 0000000180009270     JPLISAgent.obj
 0002:00002288       $unwind$getObjectArrayFromClasses 0000000180009288     JPLISAgent.obj
 0002:00002288       $unwind$invokeJavaAgentMainMethod 0000000180009288     JPLISAgent.obj
 0002:000022a0       $unwind$commonGetClassList 00000001800092a0     JPLISAgent.obj
 0002:000022b0       $unwind$getModuleObject    00000001800092b0     JPLISAgent.obj
 0002:000022c8       $unwind$JPLISAssertCondition 00000001800092c8     JPLISAssert.obj
 0002:000022c8       $unwind$JPLISAssertConditionWithMessage 00000001800092c8     JPLISAssert.obj
 0002:000022d8       $unwind$readAttributes     00000001800092d8     JarFacade.obj
 0002:000022e4       $unwind$freeAttributes     00000001800092e4     JarFacade.obj
 0002:000022f0       $unwind$createThrowable    00000001800092f0     JavaExceptions.obj
 0002:0000230c       $unwind$throwThrowable     000000018000930c     JavaExceptions.obj
 0002:0000230c       $unwind$deallocate         000000018000930c     Utilities.obj
 0002:00002314       $unwind$mapThrownThrowableIfNecessary 0000000180009314     JavaExceptions.obj
 0002:00002314       $unwind$validatePathChars  0000000180009314     PathCharsValidator.obj
 0002:00002314       $unwind$_DllMainCRTStartup 0000000180009314     MSVCRT:dll_dllmain.obj
 0002:00002324       $unwind$initialize         0000000180009324     PathCharsValidator.obj
 0002:00002324       $unwind$isInstanceofClassName 0000000180009324     Utilities.obj
 0002:0000233c       $unwind$tryToAcquireReentrancyToken 000000018000933c     Reentrancy.obj
 0002:00002350       $unwind$allocate           0000000180009350     Utilities.obj
 0002:0000235c       $unwind$__GSHandlerCheckCommon 000000018000935c     MSVCRT:gshandler.obj
 0002:00002368       $xdatasym                  0000000180009368     MSVCRT:amdsecgs.obj
 0002:0000236c       $unwind$?dllmain_crt_process_attach@@YAHQEAUHINSTANCE__@@QEAX@Z 000000018000936c     MSVCRT:dll_dllmain.obj
 0002:000023a8       $unwind$?fin$0@?0??dllmain_crt_process_attach@@YAHQEAUHINSTANCE__@@QEAX@Z@4HA 00000001800093a8     MSVCRT:dll_dllmain.obj
 0002:000023a8       $unwind$?fin$0@?0??dllmain_crt_process_detach@@YAH_N@Z@4HA 00000001800093a8     MSVCRT:dll_dllmain.obj
 0002:000023a8       $unwind$?fin$1@?0??dllmain_crt_process_detach@@YAH_N@Z@4HA 00000001800093a8     MSVCRT:dll_dllmain.obj
 0002:000023b0       $unwind$?dllmain_crt_process_detach@@YAH_N@Z 00000001800093b0     MSVCRT:dll_dllmain.obj
 0002:00002404       $unwind$?dllmain_dispatch@@YAHQEAUHINSTANCE__@@KQEAX@Z 0000000180009404     MSVCRT:dll_dllmain.obj
 0002:0000242c       $unwind$?filt$0@?0??dllmain_dispatch@@YAHQEAUHINSTANCE__@@KQEAX@Z@4HA 000000018000942c     MSVCRT:dll_dllmain.obj
 0002:00002434       $unwind$__report_gsfailure 0000000180009434     MSVCRT:gs_report.obj
 0002:0000243c       $unwind$capture_previous_context 000000018000943c     MSVCRT:gs_report.obj
 0002:00002448       $unwind$__security_init_cookie 0000000180009448     MSVCRT:gs_support.obj
 0002:00002454       $unwind$__scrt_is_nonwritable_in_current_image 0000000180009454     MSVCRT:utility.obj
 0002:00002474       $unwind$__scrt_is_nonwritable_in_current_image$filt$0 0000000180009474     MSVCRT:utility.obj
 0002:0000247c       $unwind$__scrt_fastfail    000000018000947c     MSVCRT:utility_desktop.obj
 0002:0000248c       $unwind$__isa_available_init 000000018000948c     MSVCRT:cpu_disp.obj
 0002:000024a0       $xdatasym                  00000001800094a0     MSVCRT:guard_dispatch.obj
 0002:000024a8       $xdatasym                  00000001800094a8     MSVCRT:guard_xfg_dispatch.obj
 0002:000024b0       .edata                     00000001800094b0     instrument.exp
 0002:000024d8       rgpv                       00000001800094d8     instrument.exp
 0002:00002518       rgszName                   0000000180009518     instrument.exp
 0002:00002558       rgwOrd                     0000000180009558     instrument.exp
 0002:00002578       szName                     0000000180009578     instrument.exp
 0002:00002587       $N00001                    0000000180009587     instrument.exp
 0002:00002596       $N00002                    0000000180009596     instrument.exp
 0002:000025a3       $N00003                    00000001800095a3     instrument.exp
 0002:000025b2       $N00004                    00000001800095b2     instrument.exp
 0002:000025f5       $N00005                    00000001800095f5     instrument.exp
 0002:00002632       $N00006                    0000000180009632     instrument.exp
 0002:0000266f       $N00007                    000000018000966f     instrument.exp
 0002:000026a6       $N00008                    00000001800096a6     instrument.exp
 0002:000026e1       $N00009                    00000001800096e1     instrument.exp
 0002:00002728       $N00010                    0000000180009728     instrument.exp
 0002:00002758       $N00011                    0000000180009758     instrument.exp
 0002:0000278b       $N00012                    000000018000978b     instrument.exp
 0002:000027c4       $N00013                    00000001800097c4     instrument.exp
 0002:00002800       $N00014                    0000000180009800     instrument.exp
 0002:0000284a       $N00015                    000000018000984a     instrument.exp
 0002:00002885       $N00016                    0000000180009885     instrument.exp
 0002:00002b94       .idata$6                   0000000180009b94     java:java.dll
 0002:00002bb4       .idata$6                   0000000180009bb4     jli:jli.dll
 0002:00002be2       .idata$6                   0000000180009be2     jvm:jvm.dll
 0002:00002dae       .idata$6                   0000000180009dae     kernel32:KERNEL32.dll
 0002:00002e1c       .idata$6                   0000000180009e1c     vcruntime:VCRUNTIME140.dll
 0002:00002f62       .idata$6                   0000000180009f62     ucrt:api-ms-win-crt-heap-l1-1-0.dll
 0002:00002f82       .idata$6                   0000000180009f82     ucrt:api-ms-win-crt-convert-l1-1-0.dll
 0002:00002fa4       .idata$6                   0000000180009fa4     ucrt:api-ms-win-crt-stdio-l1-1-0.dll
 0002:00002fc4       .idata$6                   0000000180009fc4     ucrt:api-ms-win-crt-string-l1-1-0.dll
 0002:00002fe6       .idata$6                   0000000180009fe6     ucrt:api-ms-win-crt-runtime-l1-1-0.dll
 0003:00000040       sFallbackInternalError     000000018000b040     JavaExceptions.obj
 0003:00000048       L_HEX                      000000018000b048     PathCharsValidator.obj
 0003:00000050       H_HEX                      000000018000b050     PathCharsValidator.obj
 0003:00000058       L_PATH                     000000018000b058     PathCharsValidator.obj
 0003:00000060       H_PATH                     000000018000b060     PathCharsValidator.obj
 0003:00000068       ?__proc_attached@@3HA      000000018000b068     MSVCRT:dll_dllmain.obj
 0003:00000070       GS_ExceptionRecord         000000018000b070     MSVCRT:gs_report.obj
 0003:00000110       GS_ContextRecord           000000018000b110     MSVCRT:gs_report.obj
 0003:00000608       ?is_initialized_as_dll@@3_NA 000000018000b608     MSVCRT:utility.obj
 0003:00000609       ?module_local_atexit_table_initialized@@3_NA 000000018000b609     MSVCRT:utility.obj
 0003:00000610       ?module_local_atexit_table@@3U_onexit_table_t@@A 000000018000b610     MSVCRT:utility.obj
 0003:00000628       ?module_local_at_quick_exit_table@@3U_onexit_table_t@@A 000000018000b628     MSVCRT:utility.obj
 0005:00000060       $R000000                   000000018000d060     instrument.dll.res
